:040000008A015428F5
:08000800F900F90E030EFA00E5
:10001000040EFB000A0EFC008A110A12A028AE286A
:10002000E128FA2804290D294D2961296F2A7D2A02
:100030009A2ABC2ADE2A362BCF2B442CAA2C392D07
:10004000AF2D782EDF2EF72F8A150A125A288A151F
:100050000A12CB288A150A12C42A8A150A12052BFD
:100060008A150A127E2B8A150A120D2C8A150A127D
:100070007E2D8A150A12862D8A150A121F2F8A15BF
:100080000A12322F8A150A128E2F8A150A12DE2FB3
:100090008A110A160F288A110A16EE288A110A16E2
:1000A00015298A110A163E2A0730831603139F006A
:1000B000C03081008312C501AC010B30B7000A309B
:1000C000B4000C30BB000D30C2000E30C4000F3045
:1000D000C900B301CC01AA01CB01CE010130BF00A0
:1000E0000230A9000330AE000430BE000530B80075
:1000F0000630CA000730B2000830B1000930BD0038
:10010000BC010130A100C801A201A001B001A701FA
:10011000A601A401C301C701B60136208A110A1243
:1001200021208A110A121B208A110A124B208A11DF
:100130000A121D208A110A121C208A110A129F28F5
:100140008B1CA6288B1019208A110A127C0E8A009B
:100150007B0E84007A0E8300790E090083168316C5
:1001600003130708C039870083120230FD001820EE
:100170008A110A12333083120313D30012208A111A
:100180000A12323083120313D30012208A110A128A
:100190002C3083120313D30012208A110A12063066
:1001A00083120313D30012208A110A120C30831217
:1001B0000313D30012208A110A1210208A110A1286
:1001C0000800013083120313D30012208A110A128F
:1001D0000130FD0018208A110A1202308312031325
:1001E000D30012208A110A120130FD0018208A1152
:1001F0000A120800831203135208D4001030D500ED
:1002000013208A110A120800831203135308D40022
:10021000D50113208A110A1208008312031354080F
:10022000F200F20CF20CF20C720C0F390F3955047B
:10023000D6000708C0395604D60087000130FD00FB
:1002400018208A110A128312031387160130FD0049
:1002500018208A110A1283120313871254080F39C7
:100260005504D6000708C0395604D600870001306F
:10027000FD0018208A110A12831203138716013019
:10028000FD0018208A110A1283120313871201300D
:10029000FD0018208A110A12080083120313D808DF
:1002A000031D55298030D8005729C030D800F201ED
:1002B000580857070318F20AD30012208A110A12AD
:1002C00008000830F200F3010830F400F501831251
:1002D00003135908F6000310F61B0314F50D6430E0
:1002E000F50203187529F5070310F60DF40B6B29B9
:1002F0007608F4000310F41B0314F30D0A30F30224
:1003000003188429F3070310F40DF20B7A297308FC
:10031000FF39003C0319F129F2013030F3000830B5
:10032000F400F5010830F600F7015908F800031051
:10033000F81B0314F70D6430F7020318A129F7071F
:100340000310F80DF60B97297808F6000310F61B3A
:100350000314F50D0A30F5020318B029F507031050
:10036000F60DF40BA629750873070318F20AD400DA
:100370001030D50013208A110A12F2013030F30038
:100380000830F400F5010830F600F701831203137A
:100390005908F8000310F81B0314F70D0A30F70290
:1003A0000318D429F7070310F80DF60BCA297808AB
:1003B000F6000310F61B0314F50D0A30F5020318BE
:1003C000E329F5070310F60DF40BD9297508730717
:1003D0000318F20AD4001030D50013208A110A1233
:1003E0004D2A0830F200F3010830F400F5018312C1
:1003F00003135908F6000310F61B0314F50D0A3019
:10040000F5020318052AF5070310F60DF40BFB2976
:100410007608F4000310F41B0314F30D0A30F30202
:100420000318142AF3070310F40DF20B0A2A7308B9
:10043000FF39003C03194D2AF2013030F300083037
:10044000F400F5010830F600F7015908F800031030
:10045000F81B0314F70D0A30F7020318312AF707C7
:100460000310F80DF60B272A7808F6000310F61B88
:100470000314F50D0A30F5020318402AF50703109E
:10048000F60DF40B362A750873070318F20AD40028
:100490001030D50013208A110A12F2013030F30017
:1004A0000830F400F501831203135908F600031015
:1004B000F61B0314F50D0A30F5020318612AF5073F
:1004C0000310F60DF40B572A750873070318F20A88
:1004D000D4001030D50013208A110A1208008312AC
:1004E0000313DB015A0803178D0083168C130C14B9
:1004F00083120C080313DB000800831603170C0893
:100500000239023C031D852A7D2A831203135C08ED
:1005100003178D0003135D0803178C0083168C13DB
:100520000C158B1355308D00AA308D008C148B1751
:100530000C110800B930FE000000000000000000AF
:1005400000000000000000000000000000000000AB
:10055000000000000000000000000000000000009B
:1005600000000000000000000000FE0B9D2A0000BB
:10057000FD0B9A2A00000800F001831203132708DC
:10058000013E0318F00AA700F0014708013E0318D6
:10059000F00AC70027083602031DD22A1E208A113E
:1005A0000A12A70147083602031DDD2A30208A11EE
:1005B0000A121F208A110A12C701080083120313AE
:1005C000D7010130D80014208A110A124430831256
:1005D0000313D20011208A110A126330831203130D
:1005E000D20011208A110A12703083120313D20034
:1005F00011208A110A12743083120313D2001120C1
:100600008A110A123A3083120313D20011208A1180
:100610000A12073083120313D7000130D8001420C8
:100620008A110A12831203132A08D90015208A118D
:100630000A12831203134E08D90015208A110A12D8
:100640002C3083120313D20011208A110A12831254
:1006500003134B08D90015208A110A1283120313C1
:100660004C08D90015208A110A1208000F208A119F
:100670000A12023083120313D700D80114208A1102
:100680000A124F3083120313D20011208A110A126A
:10069000463083120313D20011208A110A12463009
:1006A00083120313D20011208A110A122030831200
:1006B0000313D20011208A110A125230831203133D
:1006C000D20011208A110A124F3083120313D20074
:1006D00011208A110A12413083120313D200112013
:1006E0008A110A12443083120313D20011208A1196
:1006F0000A12203083120313D20011208A110A1229
:10070000543083120313D20011208A110A1252307E
:1007100083120313D20011208A110A124930831266
:100720000313D20011208A110A12503083120313CE
:10073000D20011208A110A12063083120313D70047
:100740000130D80014208A110A1283120313D90130
:1007500015208A110A12013083120313D9001520C3
:100760008A110A12413083120313D20011208A1118
:100770000A12013083120313D90015208A110A12BC
:1007800083120313D90115208A110A120330FF00C6
:1007900051208A110A1210208A110A1208000B082F
:1007A000EF3990388B002A208A110A120130831207
:1007B00003132102031DE02B2D208A110A12E32BC3
:1007C0001A208A110A1220208A110A12F2014C08FA
:1007D0004B070318F20A4E07F3000318F20A7308D6
:1007E0002A07F3000318F20A7308003C0319FA2BD6
:1007F0000030FF2B7208003C0130031D0301003C58
:100800000319D32B4508023C0318072C422C033054
:1008100045020318422C83160608BF3986000130B2
:10082000003C0319192C83120608BF394038860092
:100830001E2C831203130608BF3986006430FD00A6
:1008400018208A110A12831603130608BF3986007E
:100850002F2C83120608BF3940388600342C8312AF
:1008600003130608BF3986003230FD0018208A11B4
:100870000A12F201831203134508013E0318F20A1B
:10088000C500072CD32B080083120313D701D8010E
:1008900014208A110A12503083120313D20011203F
:1008A0008A110A12613083120313D20011208A11B7
:1008B0000A12723083120313D20011208A110A1215
:1008C000743083120313D20011208A110A123A30B5
:1008D00083120313D20011208A110A120D308312E1
:1008E0000313D700D80114208A110A124B30831247
:1008F0000313D20011208A110A126D3083120313E0
:10090000D20011208A110A12733083120313D2000D
:1009100011208A110A120D3083120313D7000130FF
:10092000D80014208A110A124B3083120313D2000C
:1009300011208A110A126D3083120313D200112084
:100940008A110A12733083120313D20011208A1104
:100950000A1208000130831203132C02031DFF2C1E
:10096000F001410840070318F00A3A07F1000318A4
:10097000F00A71082507F1000318F00A71082F0723
:10098000F1000318F00A7108003C0319C92C00306B
:10099000CE2C7008003C0130031D0301003C0319FC
:1009A000D22C382D01304102C100FF304102031D1D
:1009B000FE2C0930C10001304002C000FF3040026F
:1009C000031DFE2C0930C00001303A02BA00FF308E
:1009D0003A02031DFE2C0930BA0001302502A500A1
:1009E000FF302502031DFE2C0930A50001302F0227
:1009F000AF00FF302F02031DFE2CAF01382DF00198
:100A0000831203134108013E0318F00AC1000A30A3
:100A10004102031D382DC101F0014008013E0318B9
:100A2000F00AC0000A304002031D382DF0013A08D8
:100A3000013E0318F00ABA00C0010A303A02031D51
:100A4000382DBA01F0012508013E0318F00AA5006F
:100A50000A302502031D382DA501F0012F08013EA3
:100A60000318F00AAF000A302F02031D382DAF0122
:100A700008000130831203132C02031D6C2DF001BA
:100A80004C08013E0318F00ACC000A304C02031D4A
:100A9000AE2DCC01F0014B08013E0318F00ACB004B
:100AA0000A304B02031D6B2DCB01F0014E08013EB5
:100AB0000318F00ACE000A304E02031D6B2DF00120
:100AC0002A08013E0318F00AAA00CE010A302A02C1
:100AD000031D6B2DAA01AE2DF001831203134C08E8
:100AE0004B070318F00A4E07F1000318F00A7108CB
:100AF0002A07F1000318F00A7108003C0319822D3F
:100B00000030872D7008003C0130031D0301003CBC
:100B100003198B2DAE2D01304C02CC00FF304C025E
:100B2000031DAE2D01304B02CB000930CC00FF304D
:100B30004B02031DAE2D01304E02CE000930CB001A
:100B4000FF304E02031DAE2D01302A02AA000930EB
:100B5000CE00FF302A02031DAE2DAA010800831625
:100B60000313060880388600831206088039B50012
:100B700080303502031D772E83160608BF398600A4
:100B80000130003C0319CA2D83120608BF394038D2
:100B90008600CF2D831203130608BF398600643008
:100BA000FD0018208A110A12831603130608BF39A4
:100BB0008600E02D83120608BF3940388600E52DF7
:100BC000831203130608BF39860083160313060831
:100BD00080388600831206088039B500B508031DE9
:100BE0003E2E0B08EF398B00831605080F38850061
:100BF000831205080F39AB000F302B02031D042EA2
:100C000033208A110A123F2E0E30831203132B0257
:100C1000031D0E2E39208A110A123D2E0730831231
:100C200003132B02031D182E3C208A110A123D2E9D
:100C30000C30831203132B02031D222E21208A1154
:100C40000A123D2E0B302B02031D2A2E22208A1160
:100C50000A123D2E0330831203132B02031D342E80
:100C600027208A110A123D2E0D30831203132B0206
:100C7000031D3D2E4E208A110A123F2EE52D1D2008
:100C80008A110A120130831203132C02031D652EF0
:100C90000530D700D80114208A110A12523083126D
:100CA0000313D20011208A110A1205308312031394
:100CB000D7000130D80014208A110A125230831252
:100CC0000313D20011208A110A1283160313060897
:100CD00080388600831206088039B500B508031DE8
:100CE000722E732E652E0B08EF3990388B0008009A
:100CF00010208A110A1283120313C101C001BA0124
:100D0000A501AF01C301A401A601A701831606082E
:100D1000BF3986000130003C0319942E8312060867
:100D2000BF3940388600992E831203130608BF3955
:100D300086003230FD0018208A110A128316031330
:100D40000608BF398600AA2E83120608BF3940382C
:100D50008600AF2E831203130608BF3986001E30AB
:100D6000FD0018208A110A12831603130608BF39E2
:100D700086000130003C0319C32E83120608BF39D8
:100D800040388600C82E831203130608BF39860038
:100D90003230FD0018208A110A1283160313060848
:100DA000BF398600D92E83120608BF394038860025
:100DB000DE2E831203130608BF39860008001020B8
:100DC0008A110A12443083120313D20011208A11AF
:100DD0000A12693083120313D20011208A110A12F9
:100DE000733083120313D20011208A110A12743057
:100DF00083120313D20011208A110A126130831268
:100E00000313D20011208A110A126E3083120313C9
:100E1000D20011208A110A12633083120313D20008
:100E200011208A110A12653083120313D200112097
:100E30008A110A123D3083120313D20011208A1145
:100E40000A123F3083120313D20011208A110A12B2
:100E5000073083120313D7000130D80014208A1101
:100E60000A123F3083120313D20011208A110A1292
:100E70003F3083120313D20011208A110A122C3042
:100E800083120313D20011208A110A123F308312F9
:100E90000313D20011208A110A123F308312031368
:100EA000D20011208A110A12203083120313D200BB
:100EB00011208A110A124B3083120313D200112021
:100EC0008A110A126D3083120313D20011208A1185
:100ED0000A12733083120313D20011208A110A12EE
:100EE00083120313B308031D922F23208A110A12C1
:100EF000831203132B08AA000730D7000130D80053
:100F000014208A110A12831203132A08D90015200B
:100F10008A110A12F201831203133308013E0318E7
:100F2000F20AB30001303302031DAF2F23208A11D0
:100F30000A12831203132B08CE00F2013308013E7C
:100F40000318F20AB3004E08D90015208A110A12BC
:100F50002C3083120313D20011208A110A1202309E
:100F6000831203133302031DC72F23208A110A1291
:100F7000831203132B08CB00F2013308013E031840
:100F8000F20AB3004B08D90015208A110A12033067
:100F9000831203133302031DDF2F23208A110A1249
:100FA000831203132B08CC00F2013308013E03180F
:100FB000F20AB3004C08D90015208A110A12043035
:100FC0008312031333020318E62F702F83120313C7
:100FD000B3010230FF0051208A110A128312031359
:100FE000A101C501B90110208A110A120800831657
:100FF0000313060880388600831206088039B5007E
:101000008A150A12803035028A150A12031D5628E5
:1010100083160608BF3986000130003C03191628E4
:1010200083120608BF39403886001B288312031339
:101030000608BF3986006430FD008A110A121820A4
:101040008A150A12831603130608BF3986002E2854
:1010500083120608BF3940388600332883120313F1
:101060000608BF398600831606088038860083127A
:1010700006088039B500B508031D542883160508F5
:101080000F388500831205080F39AB008A110A1248
:1010900024208A150A122B08093C8A110A12031C03
:1010A000F72F8A150A125928332859288A110A124B
:1010B000F72F080083120313AB08031D62283F08B3
:1010C000AB00CA2801302B02031D69282908AB0098
:1010D000CA2802302B02031D70282E08AB00CA2834
:1010E00003302B02031D77284908AB00CA280430BF
:1010F0002B02031D7E283E08AB00CA2805302B02B8
:10110000031D85283808AB00CA2806302B02031DB2
:101110008C284A08AB00CA2807302B02031D9328ED
:101120004408AB00CA2808302B02031D9A28320855
:10113000AB00CA2809302B02031DA1283108AB00DF
:10114000CA280A302B02031DA8283D08AB00CA2874
:101150000B302B02031DAF284208AB00CA280C300D
:101160002B02031DB6283408AB00CA280D302B0211
:10117000031DBD283C08AB00CA280E302B02031DFE
:10118000C4283708AB00CA280F302B02031DCA2819
:101190003B08AB00080083120313B3018A110A1243
:1011A00010208A150A12433083120313D2008A11C9
:1011B0000A1211208A150A12413083120313D20039
:1011C0008A110A1211208A150A124C308312031355
:1011D000D2008A110A1211208A150A123D30831298
:1011E0000313D2008A110A1211208A150A128312DF
:1011F00003132008D9008A110A1215208A150A1231
:10120000831203132208D9008A110A1215208A15A5
:101210000A12831203134808D9008A110A121520F2
:101220008A150A12203083120313D2008A110A127F
:1012300011208A150A124D3083120313D2008A112D
:101240000A1211208A150A126F3083120313D2007A
:101250008A110A1211208A150A12643083120313AC
:10126000D2008A110A1211208A150A1269308312DB
:101270000313D2008A110A1211208A150A1266304D
:1012800083120313D2008A110A1211208A150A123E
:101290003F3083120313D2008A110A1211208A15DB
:1012A0000A12023083120313D7000130D8008A11CA
:1012B0000A1214208A150A12013083120313D9006E
:1012C0008A110A1215208A150A123D30831203135F
:1012D000D2008A110A1211208A150A124F30831285
:1012E0000313D2008A110A1211208A150A127530CE
:1012F00083120313D2008A110A1211208A150A12CE
:10130000693083120313D2008A110A1211208A1540
:101310000A12203083120313D2008A110A121120FC
:101320008A150A12203083120313D2008A110A127E
:1013300011208A150A12023083120313D9008A1170
:101340000A1215208A150A123D3083120313D200A7
:101350008A110A1211208A150A124E3083120313C1
:10136000D2008A110A1211208A150A126F308312D4
:101370000313D2008A110A1211208A150A126E3044
:1013800083120313D2008A110A1211208A110A1241
:1013900023208A150A12831203132B083F02031D10
:1013A000B62A8A110A1210208A150A1243308312B3
:1013B0000313D2008A110A1211208A150A12413031
:1013C00083120313D2008A110A1211208A150A12FD
:1013D0004C3083120313D2008A110A1211208A158D
:1013E0000A123D3083120313D2008A110A1211200F
:1013F0008A150A1283120313B308031D162A8A11D1
:101400000A1223208A150A12831203132B08A00044
:10141000D9008A110A1215208A150A12F2018312C4
:1014200003133308013E0318F20AB30001303302FC
:10143000031D312A8A110A1223208A150A128312E7
:1014400003132B08A200D9008A110A1215208A154D
:101450000A12F201831203133308013E0318F20A41
:10146000B30002303302031D4C2A8A110A122320D2
:101470008A150A12831203132B08C800D9008A1197
:101480000A1215208A150A12F20183120313330877
:10149000013E0318F20AB300033033020318512A45
:1014A000FA29F2010930F400831203132008F30033
:1014B00064300310F20CF30C0318F207F40B5A2AF1
:1014C0007308F300F4010930F6002208F5000A3031
:1014D0000310F40CF50C0318F407F60B692A7508D1
:1014E000F3070318F40A7408F20773084807F300B7
:1014F0000318F20A7308B600B301A701A601A401FC
:10150000C301C701C601CD01A801DC014808DD0007
:101510008A110A1217208A150A1201308312031346
:10152000DC002208DD008A110A1217208A150A122F
:10153000023083120313DC002008DD008A110A1236
:1015400017208A150A12033083120313DC003608B1
:10155000DD008A110A1217208A150A120230FF00D4
:101560008A110A1251208A150A12BE2A8312031305
:101570002B082902031DBD2ABE2AC6298A110A1278
:1015800010208A150A120800063083120313D700B0
:10159000D8018A110A1214208A150A128312031321
:1015A0002F08D9008A110A1215208A150A128312EF
:1015B00003132508D9008A110A1215208A150A1268
:1015C000831203133A08D9008A110A1215208A15CA
:1015D0000A122C3083120313D2008A110A1211202E
:1015E0008A150A12831203134008D9008A110A12BD
:1015F00015208A150A12831203134108D9008A1193
:101600000A1215208A150A12080083120313D70143
:101610000130D8008A110A1214208A150A12543097
:1016200083120313D2008A110A1211208A150A129A
:101630004F3083120313D2008A110A1211208A1527
:101640000A12543083120313D2008A110A12112095
:101650008A150A12203083120313D2008A110A124B
:1016600011208A150A123A3083120313D2008A110C
:101670000A1211208A150A12063083120313D700AA
:101680000130D8008A110A1214208A150A12831216
:1016900003132308D9008A110A1215208A150A1289
:1016A000831203132D08D9008A110A1215208A15F6
:1016B0000A12831203135108D9008A110A12152045
:1016C0008A150A122C3083120313D2008A110A12CF
:1016D00011208A150A12831203134F08D9008A11A8
:1016E0000A1215208A150A12831203135008D90012
:1016F0008A110A1215208A150A1208000130831275
:1017000003132C02031DD32BF00150084F070318BD
:10171000F00A5107F1000318F00A71082D07F100D3
:101720000318F00A71082307F1000318F00A710882
:10173000003C03199D2B0030A22B7008003C0130A7
:10174000031D0301003C0319A62B0C2C0130500291
:10175000D000FF305002031DD22B01304F02CF00CA
:101760000930D000FF304F02031DD22B013051024F
:10177000D1000930CF00FF305102031DD22B0130C0
:101780002D02AD000930D100FF302D02031DD22BF8
:1017900001302302A3000930AD00FF305002031DC9
:1017A000D22BA3010C2CF001831203135008013E2D
:1017B0000318F00AD0000A305002031D0C2CD0018F
:1017C000F0014F08013E0318F00ACF000A304F0223
:1017D000031D0C2CF0015108013E0318F00AD10042
:1017E000CF010A305102031D0C2CD101F0012D084C
:1017F000013E0318F00AAD000A302D02031D0C2C27
:10180000AD01F0012308013E0318F00AA3000A30DD
:101810002302031D0C2CA30108008A110A121020B8
:101820008A150A12523083120313D2008A110A1247
:1018300011208A150A12413083120313D2008A1133
:101840000A1211208A150A125A3083120313D20089
:101850008A110A1211208A150A12203083120313EA
:10186000D2008A110A1211208A150A1254308312EA
:101870000313D2008A110A1211208A150A124F305E
:1018800083120313D2008A110A1211208A150A1238
:10189000543083120313D2008A110A1211208A15C0
:1018A0000A12413083120313D2008A110A12112046
:1018B0008A150A124C3083120313D2008A110A12BD
:1018C00011208A150A1283120313D7010130D800A0
:1018D0008A110A1214208A150A124F308312031338
:1018E000D2008A110A1211208A150A127530831249
:1018F0000313D2008A110A1211208A150A126930C4
:1019000083120313D2008A110A1211208A150A12B7
:101910003D3083120313D2008A110A1211208A1556
:101920000A12413083120313D2008A110A121120C5
:101930008A150A12063083120313D7000130D8002B
:101940008A110A1214208A150A124E3083120313C8
:10195000D2008A110A1211208A150A126F308312DE
:101960000313D2008A110A1211208A150A126E304E
:1019700083120313D2008A110A1211208A150A1247
:101980003D3083120313D2008A110A1211208A15E6
:101990000A12433083120313D2008A110A12112053
:1019A0008A150A12831603130608803886008312EC
:1019B00006088039B500B508031DDF2CE02CD22CB9
:1019C0008316060880388600831206088039B50021
:1019D00080303502031D7C2D831605080F388500E5
:1019E000831205080F39AB000C302B02031D342D78
:1019F000A801CD01C601C701D001CF01D101AD01C0
:101A0000A30183160608BF3986000130003C031984
:101A10000F2D83120608BF3940388600142D83121B
:101A200003130608BF3986003230FD008A110A12FE
:101A300018208A150A12831603130608BF39860078
:101A4000272D83120608BF39403886002C2D8312BB
:101A500003130608BF3986003230FD008A110A12CE
:101A600018208A150A123C2D0F30831203132B0203
:101A7000031D3B2D3C2DE02C831603130608BF39B4
:101A800086000130003C03194B2D83120608BF3934
:101A900040388600502D831203130608BF39860094
:101AA0003230FD008A110A1218208A150A12831694
:101AB00003130608BF398600632D83120608BF3959
:101AC00040388600682D831203130608BF3986004C
:101AD0008A110A1210208A150A12831603130608A7
:101AE00080388600831206088039B500B508031DCA
:101AF0007A2D7D2D6D2D7D2DE02C08008312031392
:101B0000D001CF01D101AD01A30108008A110A1251
:101B100010208A150A1283120313D7010130D8004E
:101B20008A110A1214208A150A1232308312031302
:101B3000D2008A110A1211208A150A123D3083122E
:101B40000313D2008A110A1211208A150A1250308A
:101B500083120313D2008A110A1211208A150A1265
:101B6000413083120313D2008A110A1211208A1500
:101B70000A12553083120313D2008A110A1211205F
:101B80008A150A12533083120313D2008A110A12E3
:101B900011208A150A12453083120313D2008A11CC
:101BA0000A1211208A150A1283120313D701D801D1
:101BB0008A110A1214208A150A1231308312031373
:101BC000D2008A110A1211208A150A123D3083129E
:101BD0000313D2008A110A1211208A150A125230F8
:101BE00083120313D2008A110A1211208A150A12D5
:101BF000453083120313D2008A110A1211208A156C
:101C00000A12563083120313D2008A110A121120CD
:101C10008A150A12453083120313D2008A110A1260
:101C200011208A150A12523083120313D2008A112E
:101C30000A1211208A150A12533083120313D2009C
:101C40008A110A1211208A150A12453083120313D1
:101C5000D2008A110A1211208A110A1223208A1531
:101C60000A12831203132B083F02031D642EAC08D3
:101C7000031D3D2E0130AC003E2EAC0101302C0284
:101C8000031D522E8A110A1242208A150A120130AF
:101C9000FF008A110A1251208A110A1210208A1597
:101CA0000A12642E8A110A1242208A110A12452051
:101CB0008A150A120130FF008A110A1251208A1176
:101CC0000A1210208A150A12831203132B08290204
:101CD000031D122F8A110A1210208A110A122A20BB
:101CE0008A110A121D208A150A1283120313D701C2
:101CF0000130D8008A110A1214208A150A122030E5
:101D000083120313D2008A110A1211208A150A12B3
:101D1000203083120313D2008A110A1211208A156F
:101D20000A12203083120313D2008A110A121120E2
:101D30008A150A12203083120313D2008A110A1264
:101D400011208A150A12203083120313D2008A113F
:101D50000A1211208A150A12203083120313D200AE
:101D60008A110A1211208A150A12503083120313A5
:101D7000D2008A110A1211208A150A1241308312E8
:101D80000313D2008A110A1211208A150A12553043
:101D900083120313D2008A110A1211208A150A1223
:101DA000533083120313D2008A110A1211208A15AC
:101DB0000A12453083120313D2008A110A1211202D
:101DC0008A150A12203083120313D2008A110A12D4
:101DD00011208A150A12203083120313D2008A11AF
:101DE0000A1211208A150A12203083120313D2001E
:101DF0008A110A1211208A150A1220308312031345
:101E0000D2008A110A1211208A150A122030831278
:101E10000313D2008A110A1211208A110A123F20DC
:101E20008A150A122B083802031D192F8A110A126B
:101E300048208A110A1210208A150A1208008312FB
:101E40000313A108031D272F0130A1002C2F0130FF
:101E50002102031D2C2FA1018A110A1210208A15BC
:101E60000A1208000330FF008A110A1251208A1555
:101E70000A12831603130608BF3986000130003C9E
:101E80000319482F83120608BF39403886004D2FAA
:101E9000831203130608BF398600FF30FD008A1144
:101EA0000A1218208A150A129130FD008A110A12AE
:101EB00018208A150A12831603130608BF398600F4
:101EC000672F83120608BF39403886006C2F8312B3
:101ED00003130608BF39860083160608803886007B
:101EE000831206088039B50080303502031D792F32
:101EF0007A2F322F8A110A1210208A150A1283169D
:101F00000313060880388600831206088039B5005E
:101F1000B508031D8C2F8D2F7F2F08008A110A1200
:101F200010208A150A12043083120313D7000130DF
:101F3000D8008A110A1214208A150A12523083120C
:101F40000313D2008A110A1211208A150A12453091
:101F500083120313D2008A110A1211208A150A1261
:101F6000563083120313D2008A110A1211208A15E7
:101F70000A12453083120313D2008A110A1211206B
:101F80008A150A12523083120313D2008A110A12E0
:101F900011208A150A12533083120313D2008A11BA
:101FA0000A1211208A150A12453083120313D20037
:101FB0008A110A1211208A150A12080005308312AC
:101FC0000313D700D8018A110A1214208A150A12A5
:101FD000533083120313D2008A110A1211208A157A
:101FE0000A12543083120313D2008A110A121120EC
:101FF0008A150A124F3083120313D2008A110A1273
:1020000011208A110A165030831203138A110A16FE
:10201000D2008A110A1211208A110A16080004300F
:1020200083120313DA008A110A1216208A110A1683
:10203000C1000530DA008A110A1216208A110A1628
:10204000C0000630DA008A110A1216208A110A1618
:10205000BA000730DA008A110A1216208A110A160D
:10206000A5000830DA008A110A1216208A110A1611
:10207000AF000930DA008A110A1216208A110A16F6
:10208000D0000A30DA008A110A1216208A110A16C4
:10209000CF000B30DA008A110A1216208A110A16B4
:1020A000D1000C30DA008A110A1216208A110A16A1
:1020B000AD000D30DA008A110A1216208A110A16B4
:1020C000A3000E30DA008A110A1216208A110A16AD
:1020D000CC000F30DA008A110A1216208A110A1673
:1020E000CB001030DA008A110A1216208A110A1663
:1020F000CE001130DA008A110A1216208A110A164F
:10210000AA008A110A1210208A110A1605308312B9
:102110000313D700D8018A110A1214208A110A1653
:10212000523083120313D2008A110A1211208A112D
:102130000A16453083120313D2008A110A121120A5
:102140008A110A16533083120313D2008A110A121D
:1021500011208A110A16543083120313D2008A11F7
:102160000A1211208A110A164F3083120313D2006B
:102170008A110A1211208A110A165230831203138F
:10218000D2008A110A1211208A110A16073083120E
:102190000313D7000130D8008A110A1214208A11C3
:1021A0000A164F3083120313D2008A110A1211202B
:1021B0008A110A164B3083120313D2008A110A12B5
:1021C00011208A110A160130FF008A110A125120CB
:1021D0008A110A1210208A110A16080083120313AA
:1021E000DA018A110A1216208A110A16C800013073
:1021F000DA008A110A1216208A110A16A200023089
:10220000DA008A110A1216208A110A16A000033079
:10221000DA008A110A1216208A110A16B6008A11EB
:102220000A1248208A110A16080004308312031388
:10223000DC004108DD008A110A1217208A110A16F3
:10224000053083120313DC004008DD008A110A12F6
:1022500017208A110A16063083120313DC003A088D
:10226000DD008A110A1217208A110A16073083121C
:102270000313DC002508DD008A110A1217208A11D9
:102280000A16083083120313DC002F08DD008A11C0
:102290000A1217208A110A16093083120313DC0070
:1022A0005008DD008A110A1217208A110A160A3016
:1022B00083120313DC004F08DD008A110A12172075
:1022C0008A110A160B3083120313DC005108DD005B
:1022D0008A110A1217208A110A160C30831203136E
:1022E000DC002D08DD008A110A1217208A110A1657
:1022F0000D3083120313DC002308DD008A110A125B
:1023000017208A110A160E3083120313DC004C08C2
:10231000DD008A110A1217208A110A160F30831263
:102320000313DC004B08DD008A110A1217208A1102
:102330000A16103083120313DC004E08DD008A11E8
:102340000A1217208A110A16113083120313DC00B7
:102350002A08DD008A110A1217208A110A12102099
:102360008A110A16033083120313D700D8018A1189
:102370000A1214208A110A16533083120313D20052
:102380008A110A1211208A110A164130831203138E
:10239000D2008A110A1211208A110A1655308312AE
:1023A0000313D2008A110A1211208A110A1656301C
:1023B00083120313D2008A110A1211208A110A16FD
:1023C000453083120313D2008A110A1211208A1198
:1023D0000A16473083120313D2008A110A12112001
:1023E0008A110A16413083120313D2008A110A128D
:1023F00011208A110A16523083120313D2008A1157
:102400000A1211208A110A16443083120313D200D3
:102410008A110A1211208A110A16453083120313F9
:10242000D2008A110A1211208A110A16073083126B
:102430000313D7000130D8008A110A1214208A1120
:102440000A164F3083120313D2008A110A12112088
:102450008A110A164B3083120313D2008A110A1212
:1024600011208A110A160130FF008A110A12512028
:102470008A110A1210208A110A160800FA30FD008B
:102480008A110A1218208A110A16FA30FD008A11E0
:102490000A1218208A110A16FA30FD008A110A124F
:1024A00018208A110A16FA30FD008A110A12182023
:0A24B0008A110A16FF0B3E2A0800ED
:00000001FF
